:020000040000FA
:04080000E4EF07F02A
:1008100003B210EF05F0F2B42BEF05F09EB033EF0A
:1008200005F09EB23BEF05F0F2A81AEF04F0F2B229
:1008300025EF04F0F2A620EF04F0F2B022EF04F06E
:1008400093EF07F0F296F290FF00CD90F2929EA007
:100850002FEF04F00101533F2FEF04F0542BAEC1F2
:10086000B2F1AFC1B3F1B0C1B4F1B1C1B5F1AAC138
:10087000AEF1ABC1AFF1ACC1B0F1ADC1B1F1A6C148
:10088000AAF1A7C1ABF1A8C1ACF1A9C1ADF1A2C158
:10089000A6F1A3C1A7F1A4C1A8F1A5C1A9F19EC168
:1008A000A2F19FC1A3F1A0C1A4F1A1C1A5F19AC178
:1008B0009EF19BC19FF19CC1A0F19DC1A1F196C188
:1008C0009AF197C19BF198C19CF199C19DF1CECF4E
:1008D00096F1CFCF97F153C198F154C199F1CF6AF6
:1008E000CE6A0101536B546B9E90CD800FBC0F8E6E
:1008F0000FBA7EEF04F00F8A93EF07F00F8C0FBE54
:10090000BAEF04F096C19AF197C19BF198C19CF19E
:1009100099C19DF19AC19EF19BC19FF19CC1A0F12B
:100920009DC1A1F19EC1A2F19FC1A3F1A0C1A4F1FB
:10093000A1C1A5F1A2C1A6F1A3C1A7F1A4C1A8F1CB
:10094000A5C1A9F1A6C1AAF1A7C1ABF1A8C1ACF19B
:10095000A9C1ADF1AAC1AEF1ABC1AFF1ACC1B0F16B
:10096000ADC1B1F1AEC1B2F1AFC1B3F1B0C1B4F13B
:10097000B1C1B5F101015E6B5F6B606B616B96514C
:100980005E2797515F2398516023995161239A51B3
:100990005E279B515F239C5160239D5161239E5193
:1009A0005E279F515F23A0516023A1516123A25173
:1009B0005E27A3515F23A4516023A5516123A65153
:1009C0005E27A7515F23A8516023A9516123AA5133
:1009D0005E27AB515F23AC516023AD516123AE5113
:1009E0005E27AF515F23B0516023B1516123B251F3
:1009F0005E27B3515F23B4516023B5516123D89072
:100A0000613360335F335E33D890613360335F337B
:100A10005E33D890613360335F335E3393EF07F01A
:100A20000392030103EE00F080517F0BE92604C01E
:100A3000EFFF802B8151805D700BD8A48B8200006A
:100A40008051815D700BD8A48B9281518019D8B4EC
:100A5000079093EF07F0F2940101453F93EF07F001
:100A6000462B93EF07F09E900101533F93EF07F061
:100A7000542B93EF07F09E92040062A140EF05F023
:100A8000077C07AC5BEF05F0C274C2B455EF05F00C
:100A9000C3CFB3F5C4CFB4F50501D890B433B333A5
:100AA000D890B433B3335CEF05F0C3CF55F1C4CF66
:100AB00056F15CEF05F0C28207B4C9EF05F047C1FB
:100AC0004BF148C14CF149C14DF14AC14EF15EC1F3
:100AD00062F15FC163F160C164F161C165F196C10A
:100AE000B6F197C1B7F198C1B8F199C1B9F19AC1FE
:100AF000BAF19BC1BBF19CC1BCF19DC1BDF19EC1CE
:100B0000BEF19FC1BFF1A0C1C0F1A1C1C1F1A2C19D
:100B1000C2F1A3C1C3F1A4C1C4F1A5C1C5F1A6C16D
:100B2000C6F1A7C1C7F1A8C1C8F1A9C1C9F1AAC13D
:100B3000CAF1ABC1CBF1ACC1CCF1ADC1CDF1AEC10D
:100B4000CEF1AFC1CFF1B0C1D0F1B1C1D1F1B2C1DD
:100B5000D2F1B3C1D3F1B4C1D4F1B5C1D5F1B3C5AC
:100B6000B5F5B4C5B6F5B5C5B7F5B6C5B8F5010167
:100B700055515B2756515C23E86A5D230E2EC9EF61
:100B800005F05CC157F15DC158F15B6B5C6B5D6B4F
:100B9000078E0201002F93EF07F03C0E006F00C19B
:100BA0000CF101C10DF102C10EF103C10FF104C13D
:100BB00010F105C111F106C112F107C113F108C10D
:100BC00014F109C115F10AC116F10BC117F134C1B5
:100BD00035F105012F51000AD8B492EF06F0050156
:100BE0002F51010AD8B41CEF06F005012F51020A5B
:100BF000D8B45DEF06F005012F51030AD8B45DEFBC
:100C000006F005012F51040AD8B45DEF06F0050186
:100C10002F51050AD8B45DEF06F005012F51060AE1
:100C2000D8B45DEF06F005012F51070AD8B45DEF87
:100C300006F02F6B92EF06F00501536727EF06F0E1
:100C4000546727EF06F0556727EF06F056672BEF3E
:100C500006F092EF06F057C500F158C501F159C5ED
:100C600002F15AC503F10101010E046F000E056F78
:100C7000000E066F000E076FC4EC1DF000C157F5A3
:100C800001C158F502C159F503C15AF5006750EF8B
:100C900006F0016750EF06F0026750EF06F00367B9
:100CA00092EF06F053C557F554C558F555C559F59B
:100CB00056C55AF50F8892EF06F00501306763EFCD
:100CC00006F092EF06F00FBE78EF06F010A07DEF71
:100CD00006F00101476774EF06F0486774EF06F00D
:100CE000496774EF06F04A6778EF06F07DEF06F08B
:100CF00007AE7DEF06F08FEF06F00501312F92EF82
:100D000006F03C0E316F302F92EF06F00101000E1D
:100D1000626FE00E636FA50E646F010E656F0501D3
:100D2000306B0F880501626B33B798EF06F0628174
:100D30000CC100F10DC101F10EC102F10FC103F1AF
:100D400010C104F111C105F112C106F113C107F17F
:100D500014C108F115C109F116C10AF117C10BF14F
:100D600035C134F100C10CF101C10DF102C10EF128
:100D700003C10FF104C110F105C111F106C112F157
:100D800007C113F108C114F109C115F10AC116F127
:100D90000BC117F134C135F101018A67D7EF06F0B5
:100DA0008B67D7EF06F08C67D7EF06F08D67DBEF28
:100DB00006F00BEF07F08EC100F18FC101F190C179
:100DC00002F191C103F10101010E046F000E056FE4
:100DD000000E066F000E076FC4EC1DF000C18EF10F
:100DE00001C18FF102C190F103C191F1006700EFE1
:100DF00007F0016700EF07F0026700EF07F00367F5
:100E00000BEF07F08AC18EF18BC18FF18CC190F18D
:100E10008DC191F10F80D57ED5BE69D0D6CF47F177
:100E2000D7CF48F145C149F1E86AE8CF4AF11090BF
:100E300047C100F148C101F149C102F14AC103F1C2
:100E400001010A0E046F000E056F000E066F000E02
:100E5000076FC4EC1DF000AF1080010154A73DEFF7
:100E600007F00F9A0F9C0F9E0101000E5E6F600E3F
:100E70005F6F3D0E606F080E616F010147BF4DEF60
:100E800007F048674DEF07F049674DEF07F04A67F5
:100E90004DEF07F0F28872EF07F0F2985E6B5F6B30
:100EA000606B616B966B976B986B996B9A6B9B6B96
:100EB0009C6B9D6B9E6B9F6BA06BA16BA26BA36BDE
:100EC000A46BA56BA66BA76BA86BA96BAA6BAB6B8E
:100ED000AC6BAD6BAE6BAF6BB06BB16BB26BB36B3E
:100EE000B46BB56BD76AD66A0101456B466B0CC112
:100EF00000F10DC101F10EC102F10FC103F110C1EA
:100F000004F111C105F112C106F113C107F114C1B9
:100F100008F115C109F116C10AF117C10BF135C16C
:100F200034F193EF07F002C0E0FF005001C0D8FF9A
:100F30001000A6B299EF07F00CC0A9FF0BC0A8FFE4
:100F4000A69EA69CA684F29E550EA76EAA0EA76E1C
:100F5000A682F28EA694A6B2ABEF07F00C2A12007E
:100F6000A96EA69EA69CA680A8500C2A1200040179
:100F70002C0E826F9CEC0AF0BFEC1EF00C50B0EC13
:100F800007F0E8CF00F10C50B0EC07F0E8CF01F12A
:100F900001AFD0EF07F00101FF0E026FFF0E036FEC
:100FA00062EC1EF02967DCEF07F00401200E826F6F
:100FB0009CEC0AF0E1EF07F004012D0E826F9CEC2F
:100FC0000AF08CEC1CF01200076A0F6A106A0F011D
:100FD0000D0EC16E860EC06E030EC26E0F01280E7E
:100FE000896E130E926E080E8A6EF30E936E8B6AE4
:100FF000900E946EF18EF19E0E6A01015B6B5C6B3C
:101000005D6B576B586BF29A0101476B486B496BEC
:101010004A6B4B6B4C6B4D6B4E6B4F6B506B516B0C
:10102000526B456B466BD76AD66A0F01280ED56E98
:10103000F28A9D90B00ECD6E01015E6B5F6B606BAE
:10104000616B626B636B646B656B666B676B686B24
:10105000696B536B546BCF6ACE6A0F9A0F9C0F9ECD
:101060009D80760ECA6E9D8202013C0E006FCC6A96
:10107000160EB0EC07F0E8CF00F1170EB0EC07F059
:10108000E8CF01F1180EB0EC07F0E8CF02F1190E2D
:10109000B0EC07F0E8CF03F1010103AF6AEF08F00D
:1010A000BFEC1EF0160E0C6E00C10BF099EC07F0B1
:1010B000170E0C6E01C10BF099EC07F0180E0C6EB8
:1010C00002C10BF099EC07F0190E0C6E03C10BF086
:1010D00099EC07F000C18AF101C18BF102C18CF1DA
:1010E00003C18DF100C18EF101C18FF102C190F1F8
:1010F00003C191F11A0EB0EC07F0E8CF00F11B0E1E
:10110000B0EC07F0E8CF01F11C0EB0EC07F0E8CF2F
:1011100002F11D0EB0EC07F0E8CF03F1010103AFBF
:10112000C0EF08F0BFEC1EF01A0E0C6E00C10BF001
:1011300099EC07F01B0E0C6E01C10BF099EC07F057
:101140001C0E0C6E02C10BF099EC07F01D0E0C6E1C
:1011500003C10BF099EC07F01A0EB0EC07F0E8CFE2
:1011600000F11B0EB0EC07F0E8CF01F11C0EB0EC63
:1011700007F0E8CF02F11D0EB0EC07F0E8CF03F165
:1011800000C192F101C193F102C194F103C195F143
:10119000240EAC6E900EAB6E240EAC6E080EB86EC4
:1011A000000EB06E1F0EAF6E0401806B816B0F01DD
:1011B000900EAB6E0F019D8A0301806B816BC26B39
:1011C0008B920AEC23F02EEC24F0E4EC21F0200EBC
:1011D000B0EC07F0E8CF2FF505012F51FF0AD8A496
:1011E000F9EF08F02F6B200E0C6E2FC50BF099EC69
:1011F00007F00501010E306F3C0E316F250EB0EC8B
:1012000007F0E8CF00F1260EB0EC07F0E8CF01F1CF
:10121000270EB0EC07F0E8CF02F1280EB0EC07F093
:10122000E8CF03F1010103AF30EF09F0BFEC1EF08E
:10123000250E0C6E00C10BF099EC07F0260E0C6E1B
:1012400001C10BF099EC07F0270E0C6E02C10BF0F8
:1012500099EC07F0280E0C6E03C10BF099EC07F027
:1012600000C153F501C154F502C155F503C156F54E
:1012700000C157F501C158F502C159F503C15AF52E
:10128000290EB0EC07F0E8CF5BF505015C515B5D22
:10129000D8A05BC55CF505012F51020A0EE181B8AB
:1012A0005DEF09F005015C2F5AEF09F05BC55CF5B5
:1012B0005DEF09F081BA6DEF24F0210EB0EC07F07C
:1012C000E8CF00F1220EB0EC07F0E8CF01F1230ED9
:1012D000B0EC07F0E8CF02F1240EB0EC07F0E8CF55
:1012E00003F1010103AFA3EF09F0BFEC1EF0210EE3
:1012F0000C6E00C10BF099EC07F0220E0C6E01C1D0
:101300000BF099EC07F0230E0C6E02C10BF099EC78
:1013100007F0240E0C6E03C10BF099EC07F0210EC0
:10132000B0EC07F0E8CF00F1220EB0EC07F0E8CF08
:1013300001F1230EB0EC07F0E8CF02F1240EB0EC7F
:1013400007F0E8CF03F100C15DF501C15EF502C110
:101350005FF503C160F51BEC21F0DDEC1FF02DEC17
:101360001FF005012F51030A12E005012F51040A55
:101370001DE005012F51050A24E005012F51060A41
:1013800032E005012F51070A38E006EF0AF0ACC53C
:1013900000F101010F0E001701010051000A36E0B3
:1013A00001010051050A32E003EF0AF0ACC500F17B
:1013B00001010F0E001701010051000A27E003EFA1
:1013C0000AF00501AC51000A21E00501AC51150AF3
:1013D0001DE00501AC51300A19E00501AC51450A88
:1013E00015E003EF0AF00501AC51000A0FE005011A
:1013F000AC51300A0BE003EF0AF00501AC51000AD2
:1014000005E003EF0AF081BA6DEF24F007900001C8
:10141000F28EF28C07B017EF1BF00FB0F8EF15F05B
:101420000FB8BCEF0FF00301805181197F0BD8B4C6
:1014300017EF1BF013EE00F081517F0BE126812B9B
:10144000E7CFE8FFE00BD8B417EF1BF023EE82F0F4
:10145000C2513F0BD926E7CFDFFFC22BDF50780AFE
:10146000D8A417EF1BF007808EC100F18FC101F1E6
:1014700090C102F191C103F10101040E046F000E4D
:10148000056F000E066F000E076FC4EC1DF000AF75
:1014900053EF0AF00101030E8E6F000E8F6F000EE6
:1014A000906F000E916F03018251720AD8B4F8EF69
:1014B00015F08251520AD8B4F8EF15F08251750A2E
:1014C000D8B4F8EF15F08251630AD8B4D3EF17F00F
:1014D0008251690AD8B4B3EF12F082517A0AD8B4B3
:1014E000C6EF13F08251490AD8B452EF12F082517C
:1014F000500AD8B470EF11F08251700AD8B4B3EF2B
:1015000011F08251540AD8B4DEEF11F08251740AFE
:10151000D8B424EF12F08251730AD8B428EF15F032
:101520008251530AD8B48DEF15F082514C0AD8B4C9
:10153000B0EF0AF008EF18F0040114EE00F080514B
:101540007F0BE12682C4E7FF802B120004010D0E01
:10155000826F9CEC0AF00A0E826F9CEC0AF012007B
:1015600003018351300AD8B46BEF0DF003018351AE
:10157000310AD8B4F1EF0DF003018351320AD8B427
:1015800041EF0EF003018351330AD8B44FEF0EF050
:1015900003018351340AD8B45DEF0EF00301835187
:1015A000350AD8B4C1EF0FF003018351360AD8B41D
:1015B000EFEF0FF003018351460AD8B420EF0FF08C
:1015C000030183514D0AD8B4E4EF0BF003018351BA
:1015D0006D0AD8B4FEEF0BF003018351490AD8B469
:1015E000EFEF10F003018351500AD8B421EF10F04F
:1015F00003018351540AD8B49AEF10F003018351C8
:10160000630AD8B41EEF0CF003018351430AD8B427
:1016100016EF0DF003018351730AD8B41CEF0CF0E0
:1016200003018351610AD8B431EF0BF003018351F8
:10163000650AD8B4B9EF0DF003018351450AD8B457
:10164000C7EF0DF003018351620AD8B4D5EF0DF056
:1016500003018351420AD8B4E3EF0DF0D8A408EF98
:1016600018F004014C0E826F9CEC0AF00401610E2C
:10167000826F9CEC0AF0DDEC1FF004012C0E826FEF
:101680009CEC0AF0BFEC1EF0ABC500F1010162EC6E
:101690001EF031C182F40401300E82279CEC0AF066
:1016A00032C182F40401300E82279CEC0AF033C16F
:1016B00082F40401300E82279CEC0AF004012C0E07
:1016C000826F9CEC0AF0BFEC1EF0ACC500F101018A
:1016D00062EC1EF031C182F40401300E82279CECD2
:1016E0000AF032C182F40401300E82279CEC0AF029
:1016F00033C182F40401300E82279CEC0AF004010D
:101700002C0E826F9CEC0AF0BFEC1EF0ADC500F110
:10171000010162EC1EF031C182F40401300E822717
:101720009CEC0AF032C182F40401300E82279CEC5A
:101730000AF033C182F40401300E82279CEC0AF0D7
:1017400004012C0E826F9CEC0AF0BFEC1EF0AEC5BB
:1017500000F1010162EC1EF031C182F40401300E8F
:1017600082279CEC0AF032C182F40401300E8227F9
:101770009CEC0AF033C182F40401300E82279CEC09
:101780000AF004012C0E826F9CEC0AF0BFEC1EF0F4
:10179000B3C500F1010162EC1EF031C182F4040115
:1017A000300E82279CEC0AF032C182F40401300E24
:1017B00082279CEC0AF033C182F40401300E8227A8
:1017C0009CEC0AF01DEF10F000EC1FF084C333F125
:1017D0000DEC1FF084EC1EF0200E0C6E00C10BF01F
:1017E00099EC07F000C12FF505012F51000A06E022
:1017F00005012F51010A02E083EC20F004014C0E98
:10180000826F9CEC0AF004014D0E826F9CEC0AF092
:1018100004012C0E826F9CEC0AF0BFEC1EF02FC569
:1018200000F162EC1EF033C182F40401300E822715
:101830009CEC0AF01DEF10F06DEF24F004014C0E4B
:10184000826F9CEC0AF00401630E826F9CEC0AF03C
:101850002DEC1FF004012C0E826F9CEC0AF033EC8F
:101860000CF01DEF10F0BFEC1EF0B1C500F101014E
:10187000003B0F0E001762EC1EF033C182F404012E
:10188000300E82279CEC0AF0B1C500F101010F0E69
:101890000101001762EC1EF033C182F40401300E26
:1018A00082279CEC0AF004012D0E826F9CEC0AF05A
:1018B000B0C500F10101003B0F0E001762EC1EF0F5
:1018C00033C182F40401300E82279CEC0AF0B0C5CB
:1018D00000F101010F0E0101001762EC1EF033C18F
:1018E00082F40401300E82279CEC0AF004012D0ED4
:1018F000826F9CEC0AF0AFC500F10101003B0F0EB6
:10190000001762EC1EF033C182F40401300E82270E
:101910009CEC0AF0AFC500F101010F0E01010017A8
:1019200062EC1EF033C182F40401300E82279CEC7D
:101930000AF00401200E826F9CEC0AF0AEC500F1A3
:101940000F0E0101001762EC1EF033C182F4040196
:10195000300E82279CEC0AF00401200E826F9CEC72
:101960000AF0ADC500F101010101003B0F0E0017A7
:1019700062EC1EF033C182F40401300E82279CEC2D
:101980000AF0ADC500F101010F0E0101001762EC74
:101990001EF033C182F40401300E82279CEC0AF061
:1019A00004013A0E826F9CEC0AF0ACC500F1010113
:1019B000003B0F0E001762EC1EF033C182F40401ED
:1019C000300E82279CEC0AF0ACC500F101010F0E2D
:1019D0000101001762EC1EF033C182F40401300EE5
:1019E00082279CEC0AF004013A0E826F9CEC0AF00C
:1019F000ABC500F10101003B0F0E001762EC1EF0B9
:101A000033C182F40401300E82279CEC0AF0ABC58E
:101A100000F101010F0E001762EC1EF033C182F4D9
:101A20000401300E82279CEC0AF0120084C3E8FF08
:101A30000F0BE83AE8CFB1F585C3E8FF0F0B0501BE
:101A4000B11387C3E8FF0F0BE83AE8CFB0F588C3BE
:101A5000E8FF0F0B0501B0138AC3E8FF0F0BE83A4C
:101A6000E8CFAFF58BC3E8FF0F0B0501AF138DC3B4
:101A7000E8FF0F0BE8CFAEF58FC3E8FF0F0BE83A96
:101A8000E8CFADF590C3E8FF0F0B0501AD1392C38E
:101A9000E8FF0F0BE83AE8CFACF593C3E8FF0F0B74
:101AA0000501AC1395C3E8FF0F0BE83AE8CFABF59F
:101AB00096C3E8FF0F0B0501AB138CEC1FF004017C
:101AC0004C0E826F9CEC0AF00401430E826F9CEC7A
:101AD0000AF028EF0CF02EEC24F0BFEC1EF02DC520
:101AE00000F162EC1EF004014C0E826F9CEC0AF0D7
:101AF0000401300E826F9CEC0AF004012C0E826F00
:101B00009CEC0AF031C182F40401300E82279CEC77
:101B10000AF032C182F40401300E82279CEC0AF0F4
:101B200033C182F40401300E82279CEC0AF00401D8
:101B30002C0E826F9CEC0AF0BFEC1EF02EC500F15B
:101B400062EC1EF031C182F40401300E82279CEC5D
:101B50000AF032C182F40401300E82279CEC0AF0B4
:101B600033C182F40401300E82279CEC0AF01DEF91
:101B700010F004014C0E826F9CEC0AF00401650E1B
:101B8000826F9CEC0AF06CEC21F01DEF10F0040168
:101B90004C0E826F9CEC0AF00401450E826F9CECA7
:101BA0000AF089EC21F01DEF10F004014C0E826F59
:101BB0009CEC0AF00401620E826F9CEC0AF0C3EC0C
:101BC00021F01DEF10F004014C0E826F9CEC0AF026
:101BD0000401420E826F9CEC0AF0A6EC21F01DEF8E
:101BE00010F004014C0E826F9CEC0AF00401310EDF
:101BF000826F9CEC0AF004012C0E826F9CEC0AF0C0
:101C000025C500F126C501F127C502F128C503F15C
:101C10000101100E046F000E056F000E066F000E1E
:101C2000076FF5EC1DF062EC1EF02EC182F404018A
:101C3000300E82279CEC0AF02FC182F40401300E92
:101C400082279CEC0AF030C182F40401300E822716
:101C50009CEC0AF031C182F40401300E82279CEC26
:101C60000AF032C182F40401300E82279CEC0AF0A3
:101C700033C182F40401300E82279CEC0AF01DEF80
:101C800010F004014C0E826F9CEC0AF00401320E3D
:101C9000826F9CEC0AF0C0EC22F01DEF10F0040102
:101CA0004C0E826F9CEC0AF00401330E826F9CECA8
:101CB0000AF01DEC23F0FBEF0DF004014C0E826FD7
:101CC0009CEC0AF00401340E826F9CEC0AF00401D3
:101CD0002C0E826F9CEC0AF000EC1FF084C32AF1FA
:101CE00085C32BF186C32CF187C32DF188C32EF158
:101CF00089C32FF18AC330F18BC331F18CC332F128
:101D00008DC333F10101296B0DEC1FF084EC1EF043
:101D1000100E046F000E056F000E066F000E076FA9
:101D2000D5EC1DF000C121F501C122F502C123F55A
:101D300003C124F5E1EC23F034C5ABF535C5ACF5B2
:101D400036C5ADF537C5AEF538C5AFF539C5B0F513
:101D50003AC5B1F533EC0CF004012C0E826F9CEC0B
:101D60000AF03BC500F13CC501F13DC502F13EC59D
:101D700003F10101000E046F000E056F010E066FE6
:101D8000000E076FF5EC1DF062EC1EF02967CBEF3B
:101D90000EF0D0EF0EF004012D0E826F9CEC0AF0D5
:101DA00030C182F40401300E82279CEC0AF031C16C
:101DB00082F40401300E82279CEC0AF004012E0EFE
:101DC000826F9CEC0AF032C182F40401300E82274B
:101DD0009CEC0AF033C182F40401300E82279CECA3
:101DE0000AF004012C0E826F9CEC0AF0BFEC1EF08E
:101DF0003FC500F140C501F132EC19F004012C0E91
:101E0000826F9CEC0AF0BFEC1EF041C500F162EC61
:101E10001EF031C182F40401300E82279CEC0AF0DE
:101E200032C182F40401300E82279CEC0AF033C1E7
:101E300082F40401300E82279CEC0AF01DEF10F0B2
:101E400000EC1FF085C32AF186C32BF187C32CF168
:101E500088C32DF189C32EF18AC32FF18BC330F1D2
:101E60008CC331F18DC332F18EC333F10101296B83
:101E70000DEC1FF084EC1EF0100E046F000E056FC9
:101E8000000E066F000E076FD5EC1DF000C129F59E
:101E900001C12AF502C12BF503C12CF53BEC22F060
:101EA00004014C0E826F9CEC0AF00401460E826F16
:101EB0009CEC0AF004012C0E826F9CEC0AF025C504
:101EC00000F126C501F127C502F128C503F1010182
:101ED000100E046F000E056F000E066F000E076FE8
:101EE000F5EC1DF062EC1EF02AC182F40401300E04
:101EF00082279CEC0AF02BC182F40401300E822769
:101F00009CEC0AF02CC182F40401300E82279CEC78
:101F10000AF02DC182F40401300E82279CEC0AF0F5
:101F20002EC182F40401300E82279CEC0AF02FC1EE
:101F300082F40401300E82279CEC0AF030C182F456
:101F40000401300E82279CEC0AF031C182F40401B6
:101F5000300E82279CEC0AF032C182F40401300E6C
:101F600082279CEC0AF033C182F40401300E8227F0
:101F70009CEC0AF01DEF10F00F981DEC23F01DEF04
:101F800010F004014C0E826F9CEC0AF00401350E37
:101F9000826F9CEC0AF004012C0E826F9CEC0AF01C
:101FA000BFEC1EF00784B5C500F1079462EC1EF08B
:101FB00031C182F40401300E82279CEC0AF032C158
:101FC00082F40401300E82279CEC0AF033C182F4C3
:101FD0000401300E82279CEC0AF01DEF10F0E0ECBB
:101FE00022F0BFEC1EF033C500F162EC1EF00401DC
:101FF0004C0E826F9CEC0AF00401360E826F9CEC52
:102000000AF004012C0E826F9CEC0AF031C182F4BC
:102010000401300E82279CEC0AF032C182F40401E4
:10202000300E82279CEC0AF033C182F40401300E9A
:1020300082279CEC0AF01DEF10F0A6EC0AF008EFE6
:1020400018F004014C0E826F9CEC0AF00401500E53
:10205000826F9CEC0AF004012C0E826F9CEC0AF05B
:1020600085C32AF186C32BF187C32CF188C32DF1D8
:1020700089C32EF18AC32FF18BC330F18CC331F1A8
:102080008DC332F18EC333F101010DEC1FF084ECEE
:102090001EF003018451530A0DE0030184514D0ADF
:1020A00038E00401780E826F9CEC0AF0A6EC0AF08E
:1020B00008EF18F00401530E826F9CEC0AF0250E15
:1020C0000C6E00C10BF099EC07F0260E0C6E01C1EE
:1020D0000BF099EC07F0270E0C6E02C10BF099EC97
:1020E00007F0280E0C6E03C10BF099EC07F000C14D
:1020F00053F501C154F502C155F503C156F500C1B0
:1021000057F501C158F502C159F503C15AF5FEEF63
:1021100010F004014D0E826F9CEC0AF0290E0C6E3B
:1021200000C10BF099EC07F000C15BF500C15CF554
:10213000FEEF10F004014C0E826F9CEC0AF00401DB
:10214000540E826F9CEC0AF004012C0E826F9CEC02
:102150000AF084C32AF185C32BF186C32CF187C30F
:102160002DF188C32EF189C32FF18AC330F18BC3BF
:1021700031F18DC332F18EC333F101010DEC1FF04B
:1021800084EC1EF00101000E046F000E056F010EBD
:10219000066F000E076FD5EC1DF0210E0C6E00C10E
:1021A0000BF099EC07F0220E0C6E01C10BF099ECCC
:1021B00007F0230E0C6E02C10BF099EC07F0240E11
:1021C0000C6E03C10BF099EC07F000C15DF501C185
:1021D0005EF502C15FF503C160F5FEEF10F004018A
:1021E0004C0E826F9CEC0AF00401490E826F9CEC4D
:1021F0000AF004012C0E826F9CEC0AF0250EB0EC64
:1022000007F0E8CF00F1260EB0EC07F0E8CF01F1BF
:10221000270EB0EC07F0E8CF02F1280EB0EC07F083
:10222000E8CF03F162EC1EF045EC1CF00401730EE4
:10223000826F9CEC0AF004012C0E826F9CEC0AF079
:10224000BFEC1EF0290EB0EC07F0E8CF00F162EC15
:102250001EF045EC1CF00401730E826F9CEC0AF03A
:1022600004012C0E826F9CEC0AF057C500F158C592
:1022700001F159C502F15AC503F162EC1EF045ECBB
:102280001CF00401730E826F9CEC0AF004012C0E0A
:10229000826F9CEC0AF0BFEC1EF05CC500F162ECB2
:1022A0001EF045EC1CF004016D0E826F9CEC0AF0F0
:1022B00004012C0E826F9CEC0AF05DC500F15EC536
:1022C00001F15FC502F160C503F123EC18F00401D0
:1022D0002C0E826F9CEC0AF0A6EC0AF008EF18F0C6
:1022E00083C32AF184C32BF185C32CF186C32DF15E
:1022F00087C32EF188C32FF189C330F18AC331F12E
:102300008BC332F18CC333F101010DEC1FF084EC6F
:102310001EF0160E0C6E00C10BF099EC07F0170EB4
:102320000C6E01C10BF099EC07F0180E0C6E02C197
:102330000BF099EC07F0190E0C6E03C10BF099EC41
:1023400007F000C18AF101C18BF102C18CF103C118
:102350008DF100C18EF101C18FF102C190F103C175
:1023600091F152EF12F083C32AF184C32BF185C39C
:102370002CF186C32DF187C32EF188C32FF189C3B9
:1023800030F18AC331F18BC332F18CC333F10101D7
:102390000DEC1FF084EC1EF000C18AF101C18BF13D
:1023A00002C18CF103C18DF100C18EF101C18FF129
:1023B00002C190F103C191F152EF12F083C32AF1EF
:1023C00084C32BF185C32CF186C32DF187C32EF175
:1023D00088C32FF189C330F18AC331F18CC332F144
:1023E0008DC333F101010DEC1FF084EC1EF00101EF
:1023F000000E046F000E056F010E066F000E076FD2
:10240000D5EC1DF01A0E0C6E00C10BF099EC07F024
:102410001B0E0C6E01C10BF099EC07F01C0E0C6E3C
:1024200002C10BF099EC07F01D0E0C6E03C10BF00E
:1024300099EC07F000C192F101C193F102C194F14E
:1024400003C195F152EF12F083C32AF184C32BF13B
:1024500085C32CF186C32DF187C32EF188C32FF1DC
:1024600089C330F18AC331F18CC332F18DC333F1AA
:1024700001010DEC1FF084EC1EF00101000E046F51
:10248000000E056F010E066F000E076FD5EC1DF0F4
:1024900000C192F101C193F102C194F103C195F120
:1024A00052EF12F0160EB0EC07F0E8CF00F1170E65
:1024B000B0EC07F0E8CF01F1180EB0EC07F0E8CF70
:1024C00002F1190EB0EC07F0E8CF03F162EC1EF058
:1024D00045EC1CF00401730E826F9CEC0AF00401C1
:1024E0002C0E826F9CEC0AF08AC100F18BC101F1C5
:1024F0008CC102F18DC103F162EC1EF045EC1CF0C1
:102500000401730E826F9CEC0AF004012C0E826FA2
:102510009CEC0AF01A0EB0EC07F0E8CF00F11B0EAD
:10252000B0EC07F0E8CF01F11C0EB0EC07F0E8CFFB
:1025300002F11D0EB0EC07F0E8CF03F123EC18F028
:1025400004012C0E826F9CEC0AF092C100F193C141
:1025500001F194C102F195C103F123EC18F0A6EC4E
:102560000AF008EF18F00401690E826F9CEC0AF083
:1025700004012C0E826F9CEC0AF00101040E006F26
:10258000000E016F000E026F000E036F62EC1EF072
:102590002CC182F40401300E82279CEC0AF02DC17C
:1025A00082F40401300E82279CEC0AF02EC182F4E2
:1025B0000401300E82279CEC0AF02FC182F4040142
:1025C000300E82279CEC0AF030C182F40401300EF8
:1025D00082279CEC0AF031C182F40401300E82277C
:1025E0009CEC0AF032C182F40401300E82279CEC8C
:1025F0000AF033C182F40401300E82279CEC0AF009
:1026000004012C0E826F9CEC0AF00101060E006F93
:10261000000E016F000E026F000E036F62EC1EF0E1
:102620002CC182F40401300E82279CEC0AF02DC1EB
:1026300082F40401300E82279CEC0AF02EC182F451
:102640000401300E82279CEC0AF02FC182F40401B1
:10265000300E82279CEC0AF030C182F40401300E67
:1026600082279CEC0AF031C182F40401300E8227EB
:102670009CEC0AF032C182F40401300E82279CECFB
:102680000AF033C182F40401300E82279CEC0AF078
:1026900004012C0E826F9CEC0AF001011B0E006FEE
:1026A000000E016F000E026F000E036F62EC1EF051
:1026B0002CC182F40401300E82279CEC0AF02DC15B
:1026C00082F40401300E82279CEC0AF02EC182F4C1
:1026D0000401300E82279CEC0AF02FC182F4040121
:1026E000300E82279CEC0AF030C182F40401300ED7
:1026F00082279CEC0AF031C182F40401300E82275B
:102700009CEC0AF032C182F40401300E82279CEC6A
:102710000AF033C182F40401300E82279CEC0AF0E7
:1027200004012C0E826F9CEC0AF0200EF86EF76A02
:10273000F66A04010900F5CF82F49CEC0AF0090066
:10274000F5CF82F49CEC0AF00900F5CF82F49CEC02
:102750000AF00900F5CF82F49CEC0AF00900F5CFED
:1027600082F49CEC0AF00900F5CF82F49CEC0AF0AC
:102770000900F5CF82F49CEC0AF00900F5CF82F451
:102780009CEC0AF0A6EC0AF008EF18F08351630AFB
:10279000D8A408EF18F08451610AD8A408EF18F003
:1027A00085516C0AD8A408EF18F08651410A42E01E
:1027B0008651440A1BE08651420AD8B42DEF14F02A
:1027C0008651350AD8B492EF19F08651360AD8B43A
:1027D000E7EF19F08651370AD8B450EF1AF0865156
:1027E000380AD8B4AEEF1AF008EF18F00798079A35
:1027F00004017A0E826F9CEC0AF00401780E826F5D
:102800009CEC0AF00401640E826F9CEC0AF081A833
:1028100011EF14F00401550E826F9CEC0AF016EFD4
:1028200014F004014C0E826F9CEC0AF0A6EC0AF046
:1028300008EF18F00788079A04017A0E826F9CEC63
:102840000AF00401410E826F9CEC0AF00401610E53
:10285000826F9CEC0AF007EF14F00798078A0401D6
:102860007A0E826F9CEC0AF00401420E826F9CEC9F
:102870000AF00401610E826F9CEC0AF007EF14F07D
:10288000010166674BEF14F067674BEF14F0686760
:102890004BEF14F0696763EF14F04F6757EF14F0D4
:1028A000506757EF14F0516757EF14F0526763EF1A
:1028B00014F00101000E006F000E016F000E026F98
:1028C000000E036F12000101620E046F010E056F0E
:1028D000000E066F000E076F66C100F167C101F1BF
:1028E00068C102F169C103F1C4EC1DF003BFE7EF59
:1028F00014F00101000E046FA80E056F550E066F4F
:10290000020E076F66C100F167C101F168C102F1F3
:1029100069C103F166C186F167C187F168C188F1B9
:1029200069C189F1C4EC1DF003BFA0EF14F00101EF
:10293000000E866FA80E876F550E886F020E896F86
:102940000E0EB0EC07F0E8CF18F10F0EB0EC07F068
:10295000E8CF19F1100EB0EC07F0E8CF1AF1110E24
:10296000B0EC07F0E8CF1BF10DEC1DF086C104F1CF
:1029700087C105F188C106F189C107F1C4EC1DF0DA
:102980000782D1EC1CF00DEC1DF00792D1EC1CF08D
:1029900086C100F187C101F188C102F189C103F14B
:1029A0000792D1EC1CF0CC0E046FE00E056F870E81
:1029B000066F050E076FC4EC1DF000C118F101C1D0
:1029C00019F102C11AF103C11BF11FEF15F001014A
:1029D000800E006F1A0E016F060E026F000E036F5D
:1029E0004FC104F150C105F151C106F152C107F1C7
:1029F000C4EC1DF003AF00EF15F0BFEC1EF01200A9
:102A00000E0EB0EC07F0E8CF18F10F0EB0EC07F0A7
:102A1000E8CF19F1100EB0EC07F0E8CF1AF1110E63
:102A2000B0EC07F0E8CF1BF14FC100F150C101F14C
:102A300051C102F152C103F10782D1EC1CF018C15F
:102A400000F119C101F11AC102F11BC103F1120019
:102A50000401730E826F9CEC0AF004012C0E826F4D
:102A60009CEC0AF0078462C166F163C167F164C13E
:102A700068F165C169F14BC14FF14CC150F14DC1D5
:102A800051F14EC152F157C159F158C15AF1079451
:102A90004EEC15F0A6EC0AF008EF18F066C100F154
:102AA00067C101F168C102F169C103F1010162EC82
:102AB0001EF045EC1CF00401630E826F9CEC0AF0E2
:102AC00004012C0E826F9CEC0AF04FC100F150C142
:102AD00001F151C102F152C103F1010162EC1EF09A
:102AE00045EC1CF00401660E826F9CEC0AF00401B8
:102AF0002C0E826F9CEC0AF0BFEC1EF059C100F165
:102B00005AC101F1010162EC1EF045EC1CF0040118
:102B1000740E826F9CEC0AF0120010820401530EB6
:102B2000826F9CEC0AF004012C0E826F9CEC0AF080
:102B300083C32AF184C32BF185C32CF186C32DF105
:102B400087C32EF188C32FF189C330F18AC331F1D5
:102B50008BC332F18CC333F101010DEC1FF084EC17
:102B60001EF000C166F101C167F102C168F103C145
:102B700069F18EC32AF18FC32BF190C32CF191C35D
:102B80002DF192C32EF193C32FF194C330F195C36D
:102B900031F196C332F197C333F101010DEC1FF00F
:102BA00084EC1EF000C14FF101C150F102C151F19E
:102BB00003C152F100EC1FF099C32FF19AC330F119
:102BC0009BC331F19CC332F19DC333F101010DEC84
:102BD0001FF084EC1EF000C159F101C15AF14EEC16
:102BE00015F004012C0E826F9CEC0AF0FFEF15F03B
:102BF0008251520A03E10F82FFEF15F00F928251CA
:102C0000750A03E1108406EF16F010948251550AFC
:102C100003E110860DEF16F01096078410B26AEFEC
:102C200016F010A456EF16F0B6C166F1B7C167F101
:102C3000B8C168F1B9C169F1BAC16AF1BBC16BF140
:102C4000BCC16CF1BDC16DF1BEC16EF1BFC16FF110
:102C5000C0C170F1C1C171F1C2C172F1C3C173F1E0
:102C6000C4C174F1C5C175F1C6C176F1C7C177F1B0
:102C7000C8C178F1C9C179F1CAC17AF1CBC17BF180
:102C8000CCC17CF1CDC17DF1CEC17EF1CFC17FF150
:102C9000D0C180F1D1C181F1D2C182F1D3C183F120
:102CA000D4C184F1D5C185F15EEF16F062C166F141
:102CB00063C167F164C168F165C169F14BC14FF14E
:102CC0004CC150F14DC151F14EC152F157C159F1B2
:102CD00058C15AF107940FA08CEF16F001019267CA
:102CE00079EF16F0936779EF16F0946779EF16F0A5
:102CF00095677DEF16F08CEF16F040EC14F092C162
:102D000004F193C105F194C106F195C107F1C4EC3A
:102D10001DF003BFD0EF17F040EC14F00101000EDE
:102D2000046F000E056F010E066F000E076FF5ECC5
:102D30001DF010A4A3EF16F00401750E826F9CEC39
:102D40000AF0A8EF16F00401720E826F9CEC0AF0F4
:102D500004012C0E826F9CEC0AF062EC1EF02967D5
:102D6000B7EF16F00401200E826FBAEF16F00401DF
:102D70002D0E826F9CEC0AF030C182F40401300EFB
:102D800082279CEC0AF031C182F40401300E8227C4
:102D90009CEC0AF004012E0E826F9CEC0AF032C10A
:102DA00082F40401300E82279CEC0AF033C182F4D5
:102DB0000401300E82279CEC0AF004016D0E826F34
:102DC0009CEC0AF004012C0E826F9CEC0AF04FC1BF
:102DD00000F150C101F151C102F152C103F10101F1
:102DE00062EC1EF045EC1CF00401480E826F9CEC76
:102DF0000AF004017A0E826F9CEC0AF004012C0E9A
:102E0000826F9CEC0AF066C100F167C101F168C1F4
:102E100002F169C103F1010162EC1EF045EC1CF006
:102E20000401630E826F9CEC0AF004012C0E826F89
:102E30009CEC0AF066C100F167C101F168C102F1C2
:102E400069C103F101010A0E046F000E056F000E47
:102E5000066F000E076FD5EC1DF0000E046F120E0A
:102E6000056F000E066F000E076FF5EC1DF062ECAB
:102E70001EF02AC182F40401300E82279CEC0AF075
:102E80002BC182F40401300E82279CEC0AF02CC185
:102E900082F40401300E82279CEC0AF02DC182F4EA
:102EA0000401300E82279CEC0AF02EC182F404014A
:102EB000300E82279CEC0AF02FC182F40401300E00
:102EC00082279CEC0AF030C182F40401300E822784
:102ED0009CEC0AF004012E0E826F9CEC0AF031C1CA
:102EE00082F40401300E82279CEC0AF032C182F495
:102EF0000401300E82279CEC0AF033C182F40401F5
:102F0000300E82279CEC0AF00401730E826F9CEC59
:102F10000AF004012C0E826F9CEC0AF0BFEC1EF04C
:102F200059C100F15AC101F132EC19F00FB29CEF16
:102F300017F00FA0CEEF17F004012C0E826F9CEC5F
:102F40000AF0200EF86EF76AF66A04010900F5CF60
:102F500082F49CEC0AF00900F5CF82F49CEC0AF0B4
:102F60000900F5CF82F49CEC0AF00900F5CF82F459
:102F70009CEC0AF00900F5CF82F49CEC0AF0090001
:102F8000F5CF82F49CEC0AF00900F5CF82F49CECBA
:102F90000AF00900F5CF82F49CEC0AF0A6EC0AF0E6
:102FA0000F9008EF18F00401630E826F9CEC0AF09A
:102FB00004012C0E826F9CEC0AF00EEC18F0040158
:102FC0002C0E826F9CEC0AF081EC18F004012C0EA0
:102FD000826F9CEC0AF0FDEC18F004012C0E826F5D
:102FE0009CEC0AF00101F80E006FCD0E016F660E29
:102FF000026F030E036F23EC18F004012C0E826F96
:103000009CEC0AF013EC19F0A6EC0AF008EF18F0AB
:103010000301C26B0790109217EF1BF0D8900E0EB1
:10302000B0EC07F0E8CF00F10F0EB0EC07F0E8CFFE
:1030300001F1100EB0EC07F0E8CF02F1110EB0EC88
:1030400007F0E8CF03F10101000E046F000E056FD9
:10305000010E066F000E076FF5EC1DF062EC1EF01E
:103060002AC182F40401300E82279CEC0AF02BC1A5
:1030700082F40401300E82279CEC0AF02CC182F409
:103080000401300E82279CEC0AF02DC182F4040169
:10309000300E82279CEC0AF02EC182F40401300E1F
:1030A00082279CEC0AF02FC182F40401300E8227A3
:1030B0009CEC0AF030C182F40401300E82279CECB3
:1030C0000AF031C182F40401300E82279CEC0AF030
:1030D00004012E0E826F9CEC0AF032C182F40401CE
:1030E000300E82279CEC0AF033C182F40401300ECA
:1030F00082279CEC0AF004016D0E826F9CEC0AF0B2
:103100001200120EB0EC07F0E8CF00F1130EB0EC95
:1031100007F0E8CF01F1140EB0EC07F0E8CF02F1B0
:10312000150EB0EC07F0E8CF03F101010A0E046FB1
:10313000000E056F000E066F000E076FD5EC1DF038
:10314000000E046F120E056F000E066F000E076F63
:10315000F5EC1DF062EC1EF02AC182F40401300E81
:1031600082279CEC0AF02BC182F40401300E8227E6
:103170009CEC0AF02CC182F40401300E82279CECF6
:103180000AF02DC182F40401300E82279CEC0AF073
:103190002EC182F40401300E82279CEC0AF02FC16C
:1031A00082F40401300E82279CEC0AF030C182F4D4
:1031B0000401300E82279CEC0AF004012E0E826F6F
:1031C0009CEC0AF031C182F40401300E82279CECA1
:1031D0000AF032C182F40401300E82279CEC0AF01E
:1031E00033C182F40401300E82279CEC0AF0040102
:1031F000730E826F9CEC0AF012000A0EB0EC07F01E
:10320000E8CF00F10B0EB0EC07F0E8CF01F10C0EA7
:10321000B0EC07F0E8CF02F10D0EB0EC07F0E8CF0C
:1032200003F132EF19F0060EB0EC07F0E8CF00F131
:10323000070EB0EC07F0E8CF01F1080EB0EC07F094
:10324000E8CF02F1090EB0EC07F0E8CF03F132EF5E
:1032500019F00101BFEC1EF0078457C100F158C1FD
:1032600001F107940101E80E046F800E056F000E56
:10327000066F000E076FD5EC1DF0000E046F040EF4
:10328000056F000E066F000E076FF5EC1DF0880E3F
:10329000046F130E056F000E066F000E076FC4EC6F
:1032A0001DF00A0E046F000E056F000E066F000E73
:1032B000076FF5EC1DF062EC1EF00101296766EF67
:1032C00019F00401200E826F69EF19F004012D0E30
:1032D000826F9CEC0AF030C182F40401300E822728
:1032E0009CEC0AF031C182F40401300E82279CEC80
:1032F0000AF032C182F40401300E82279CEC0AF0FD
:1033000004012E0E826F9CEC0AF033C182F404019A
:10331000300E82279CEC0AF00401430E826F9CEC75
:103320000AF0120087C32AF188C32BF189C32CF15C
:103330008AC32DF18BC32EF18CC32FF18DC330F1D5
:103340008EC331F190C332F191C333F10101296B86
:103350000DEC1FF084EC1EF00101000E046F000E56
:10336000056F010E066F000E076FD5EC1DF00E0EF7
:103370000C6E00C10BF099EC07F00F0E0C6E01C142
:103380000BF099EC07F0100E0C6E02C10BF099ECEB
:1033900007F0110E0C6E03C10BF099EC07F004015D
:1033A0007A0E826F9CEC0AF004012C0E826F9CEC6A
:1033B0000AF00401350E826F9CEC0AF004012C0E19
:1033C000826F9CEC0AF00EEC18F016EF14F087C335
:1033D0002AF188C32BF189C32CF18AC32DF18BC349
:1033E0002EF18CC32FF18DC330F18EC331F190C318
:1033F00032F191C333F10101296B0DEC1FF084EC24
:103400001EF0880E046F130E056F000E066F000E7F
:10341000076FC9EC1DF0000E046F040E056F000E5F
:10342000066F000E076FD5EC1DF00101E80E046F6A
:10343000800E056F000E066F000E076FF5EC1DF095
:103440000A0E0C6E00C10BF099EC07F00B0E0C6E1F
:1034500001C10BF099EC07F00C0E0C6E02C10BF0E1
:1034600099EC07F00D0E0C6E03C10BF099EC07F010
:1034700004017A0E826F9CEC0AF004012C0E826F1C
:103480009CEC0AF00401360E826F9CEC0AF00401F9
:103490002C0E826F9CEC0AF0FDEC18F016EF14F085
:1034A00087C32AF188C32BF189C32CF18AC32DF17C
:1034B0008BC32EF18CC32FF18DC330F18FC331F14B
:1034C00090C332F191C333F101010DEC1FF084EC94
:1034D0001EF0000E046F120E056F000E066F000E38
:1034E000076FD5EC1DF001010A0E046F000E056F89
:1034F000000E066F000E076FF5EC1DF0120E0C6E3D
:1035000000C10BF099EC07F0130E0C6E01C10BF02B
:1035100099EC07F0140E0C6E02C10BF099EC07F059
:10352000150E0C6E03C10BF099EC07F004017A0E36
:10353000826F9CEC0AF004012C0E826F9CEC0AF066
:103540000401370E826F9CEC0AF004012C0E826F8E
:103550009CEC0AF081EC18F016EF14F087C32AF106
:1035600088C32BF189C32CF18AC32DF18BC32EF1B3
:103570008CC32FF18DC330F18EC331F190C332F182
:1035800091C333F10101296B0DEC1FF084EC1EF0A7
:10359000880E046F130E056F000E066F000E076F86
:1035A000C9EC1DF0000E046F040E056F000E066FCF
:1035B000000E076FD5EC1DF00101E80E046F800EC0
:1035C000056F000E066F000E076FF5EC1DF0060E7E
:1035D0000C6E00C10BF099EC07F0070E0C6E01C1E8
:1035E0000BF099EC07F0080E0C6E02C10BF099EC91
:1035F00007F0090E0C6E03C10BF099EC07F0040103
:103600007A0E826F9CEC0AF004012C0E826F9CEC07
:103610000AF00401380E826F9CEC0AF004012C0EB3
:10362000826F9CEC0AF013EC19F016EF14F081A8ED
:10363000D5EF1BF007A88EEF1BF00101800E006F85
:103640001A0E016F060E026F000E036F4BC104F1DC
:103650004CC105F14DC106F14EC107F1C4EC1DF09E
:1036600003BFD5EF1BF03FEC1CF04BC100F14CC188
:1036700001F14DC102F14EC103F10782D1EC1CF002
:1036800018C104F119C105F11AC106F11BC107F1F6
:10369000F80E006FCD0E016F660E026F030E036F02
:1036A000C4EC1DF00E0E0C6E00C10BF099EC07F08F
:1036B0000F0E0C6E01C10BF099EC07F0100E0C6EA2
:1036C00002C10BF099EC07F0110E0C6E03C10BF068
:1036D00099EC07F007840101BFEC1EF057C100F11F
:1036E00058C101F107940A0E0C6E00C10BF099EC61
:1036F00007F00B0E0C6E01C10BF099EC07F00C0EED
:103700000C6E02C10BF099EC07F00D0E0C6E03C1AC
:103710000BF099EC07F00798D5EF1BF007AAD5EF4F
:103720001BF007840101BFEC1EF057C100F158C126
:1037300001F10794060E0C6E00C10BF099EC07F036
:10374000070E0C6E01C10BF099EC07F0080E0C6E21
:1037500002C10BF099EC07F0090E0C6E03C10BF0DF
:1037600099EC07F0078462C100F163C101F164C103
:1037700002F165C103F10794120E0C6E00C10BF04B
:1037800099EC07F0130E0C6E01C10BF099EC07F0E9
:10379000140E0C6E02C10BF099EC07F0150E0C6EB6
:1037A00003C10BF099EC07F0079A040180518119CD
:1037B0007F0B0BE09EA809D014EE00F081517F0B27
:1037C000E126E750812B0F01AD6E05012F51010A53
:1037D00013E081AAFCEF1BF005012F51000A0AE05B
:1037E0000FB8FCEF1BF005013067FCEF1BF00FB8C2
:1037F000FCEF1BF06DEF24F081B811EF1CF0DDEC55
:103800001FF005012F51020A02E011EF1CF05C2F9E
:1038100011EF1CF05BC55CF50501010E306F3C0E2D
:10382000316F0AEF0AF018C100F119C101F11AC194
:1038300002F11BC103F1000E046F000E056F010EB3
:10384000066F000E076FF5EC1DF029A13EEF1CF08E
:103850002051D8B43EEF1CF018C100F119C101F19C
:103860001AC102F11BC103F1000E046F000E056FB7
:103870000A0E066F000E076FF5EC1DF01200010135
:10388000186B196B1A6B1B6B12002AC182F40401AE
:10389000300E82279CEC0AF02BC182F40401300E1A
:1038A00082279CEC0AF02CC182F40401300E82279E
:1038B0009CEC0AF02DC182F40401300E82279CECAE
:1038C0000AF02EC182F40401300E82279CEC0AF02B
:1038D0002FC182F40401300E82279CEC0AF030C123
:1038E00082F40401300E82279CEC0AF031C182F48C
:1038F0000401300E82279CEC0AF032C182F40401EC
:10390000300E82279CEC0AF033C182F40401300EA1
:1039100082279CEC0AF012002FC182F40401300EC1
:1039200082279CEC0AF030C182F40401300E822719
:103930009CEC0AF031C182F40401300E82279CEC29
:103940000AF032C182F40401300E82279CEC0AF0A6
:1039500033C182F40401300E82279CEC0AF012007D
:10396000060E116E060E126E060E136E112EB6EFB7
:103970001CF0122EB6EF1CF0132EB6EF1CF08B8449
:10398000020E116E020E126E020E136E112EC6EF93
:103990001CF0122EC6EF1CF0132EC6EF1CF08B94F9
:1039A00012000101005305E1015303E1025301E15B
:1039B000002B94EC1DF0BFEC1EF03951006F3A5112
:1039C000016F420E046F4B0E056F000E066F000E66
:1039D000076FD5EC1DF000C104F101C105F102C172
:1039E00006F103C107F118C100F119C101F11AC1B3
:1039F00002F11BC103F107B202EF1DF0C9EC1DF08B
:103A000004EF1DF0C4EC1DF000C118F101C119F163
:103A100002C11AF103C11BF11200BFEC1EF059C123
:103A200000F15AC101F1060EB0EC07F0E8CF04F145
:103A3000070EB0EC07F0E8CF05F1080EB0EC07F088
:103A4000E8CF06F1090EB0EC07F0E8CF07F1C4ECBF
:103A50001DF000C124F101C125F102C126F103C10D
:103A600027F1290E046F000E056F000E066F000E81
:103A7000076FD5EC1DF0EE0E046F430E056F000EC0
:103A8000066F000E076FC9EC1DF024C104F125C1BB
:103A900005F126C106F127C107F1D5EC1DF000C1E3
:103AA0001CF101C11DF102C11EF103C11FF1120E73
:103AB000B0EC07F0E8CF04F1130EB0EC07F0E8CF5C
:103AC00005F1140EB0EC07F0E8CF06F1150EB0ECDE
:103AD00007F0E8CF07F10D0E006F000E016F000E2A
:103AE000026F000E036FD5EC1DF0180E046F000E70
:103AF000056F000E066F000E076FF5EC1DF01CC180
:103B000004F11DC105F11EC106F11FC107F1C9EC89
:103B10001DF06A0E046F2A0E056F000E066F000E70
:103B2000076FC4EC1DF01200BF0EFA6E200E3A6F44
:103B3000396BD8900037013702370337D8B0A5EF7B
:103B40001DF03A2F9AEF1DF039073A070353D8B406
:103B500012000331070B80093F6F03390F0B010F70
:103B6000396F80EC5FF0406F390580EC5FF0405DAD
:103B7000405F396B3F33D8B0392739333FA9BAEFAB
:103B80001DF04051392712003D01E4EC1EF0D8B081
:103B90001200010103510719346FA7EC1EF0D890F1
:103BA0000751031934AF800F12000101346BCBECC5
:103BB0001EF0D8A0E1EC1EF0D8B01200B6EC1EF05A
:103BC000BFEC1EF01F0E366FF7EC1EF00B35D8B0B1
:103BD000A7EC1EF0D8A00335D8B01200362FE4EFC2
:103BE0001DF034B1CEEC1EF012000101346B045113
:103BF0000511061107110008D8A0CBEC1EF0D8A0C3
:103C0000E1EC1EF0D8B01200086B096B0A6B0B6B6D
:103C1000F7EC1EF01F0E366FF7EC1EF007510B5D30
:103C2000D8A41FEF1EF006510A5DD8A41FEF1EF0A6
:103C30000551095DD8A41FEF1EF00451085DD8A0FE
:103C400032EF1EF00451085F0551D8A0053D095F11
:103C50000651D8A0063D0A5F0751D8A0073D0B5F6B
:103C6000D8900081362F0CEF1EF034B1CEEC1EF050
:103C7000346BCBEC1EF0D890FBEC1EF007510B5DC3
:103C8000D8A44FEF1EF006510A5DD8A44FEF1EF0E6
:103C90000551095DD8A44FEF1EF00451085DD8A06E
:103CA0005EEF1EF0003F5EEF1EF0013F5EEF1EF084
:103CB000023F5EEF1EF0032BD8B4120034B1CEECFD
:103CC0001EF012000101346BCBEC1EF0D8B01200D4
:103CD00000EC1FF0200E366F003701370237033734
:103CE00011EE33F00A0E376FE7360A0EE75CD8B0F4
:103CF000E76EE552372F74EF1EF0362F6CEF1EF093
:103D000034B12981D890120001010A0E346F200EBF
:103D1000366F11EE29F03451376F0A0ED890E65203
:103D2000D8B0E726E732372F8FEF1EF00333023388
:103D300001330033362F89EF1EF0E750FF0FD8A074
:103D40000335D8B0120029B1CEEC1EF01200045198
:103D500000270551D8B0053D01270651D8B0063DD2
:103D600002270751D8B0073D032712000051086F02
:103D70000151096F02510A6F03510B6F12000101CB
:103D8000006B016B026B036B12000101046B056B8E
:103D9000066B076B12000335D8A012000351800B8D
:103DA000001F011F021F031F003FDEEF1EF0013F37
:103DB000DEEF1EF0023FDEEF1EF0032B342B032557
:103DC00012000735D8A012000751800B041F051FF1
:103DD000061F071F043FF4EF1EF0053FF4EF1EF02F
:103DE000063FF4EF1EF0072B342B07251200003797
:103DF000013702370337083709370A370B37120004
:103E00000101296B2A6B2B6B2C6B2D6B2E6B2F6B8F
:103E1000306B316B326B336B120001012A510F0B87
:103E20002A6F2B510F0B2B6F2C510F0B2C6F2D5119
:103E30000F0B2D6F2E510F0B2E6F2F510F0B2F6F5E
:103E400030510F0B306F31510F0B316F32510F0B5F
:103E5000326F33510F0B336F12008984000EC76E1F
:103E6000220EC66E9E96C69E000EC96EFF0E9EB6B0
:103E700002D0E82EFCD79E96C69E000EC96EFF0E9D
:103E80009EB602D0E82EFCD7C9CFABF59E96C69E53
:103E9000000EC96EFF0E9EB602D0E82EFCD7C9CF29
:103EA000ACF59E96C69E000EC96EFF0E9EB602D061
:103EB000E82EFCD7C9CFADF59E96C69E000EC96E02
:103EC000FF0E9EB602D0E82EFCD7C9CFAEF59E9667
:103ED000C69E000EC96EFF0E9EB602D0E82EFCD71D
:103EE000C9CFAFF59E96C69E000EC96EFF0E9EB658
:103EF00002D0E82EFCD7C9CFB0F59E96C69E000E24
:103F0000C96EFF0E9EB602D0E82EFCD7C9CFB1F520
:103F10008994E0EC21F012008984000EC76E220E15
:103F2000C66E9E96C69E800EC96EFF0E9EB602D0CD
:103F3000E82EFCD79E96C69EABC5C9FFFF0E9EB667
:103F400002D0E82EFCD79E96C69EACC5C9FFFF0ED8
:103F50009EB602D0E82EFCD79E96C69EADC5C9FF80
:103F6000FF0E9EB602D0E82EFCD79E96C69EAEC52A
:103F7000C9FFFF0E9EB602D0E82EFCD79E96C69EC5
:103F8000AFC5C9FFFF0E9EB602D0E82EFCD79E96A5
:103F9000C69EB0C5C9FFFF0E9EB602D0E82EFCD764
:103FA0009E96C69EB1C5C9FFFF0E9EB602D0E82EF2
:103FB000FCD78994E0EC21F012008984000EC76ED2
:103FC000220EC66E9E96C69E070EC96EFF0E9EB648
:103FD00002D0E82EFCD79E96C69E000EC96EFF0E3C
:103FE0009EB602D0E82EFCD7C9CFABF59E96C69EF2
:103FF000000EC96EFF0E9EB602D0E82EFCD7C9CFC8
:10400000ACF59E96C69E000EC96EFF0E9EB602D0FF
:10401000E82EFCD7C9CFADF59E96C69E000EC96EA0
:10402000FF0E9EB602D0E82EFCD7C9CFAEF589941C
:10403000E0EC21F08984000EC76E220EC66E9E96BB
:10404000C69E0F0EC96EFF0E9EB602D0E82EFCD79C
:104050009E96C69E000EC96EFF0E9EB602D0E82E3A
:10406000FCD7C9CFB3F58994E0EC21F01200898424
:10407000000EC76E220EC66E9E96C69E870EC96E35
:10408000FF0E9EB602D0E82EFCD79E96C69EABC50C
:10409000C9FFFF0E9EB602D0E82EFCD79E96C69EA4
:1040A000ACC5C9FFFF0E9EB602D0E82EFCD79E9687
:1040B000C69EADC5C9FFFF0E9EB602D0E82EFCD746
:1040C0009E96C69EAEC5C9FFFF0E9EB602D0E82ED4
:1040D000FCD78994E0EC21F089849E96C69E8F0ED1
:1040E000C96EFF0E9EB602D0E82EFCD79E96C69EE5
:1040F000B3C5C9FFFF0E9EB602D0E82EFCD7899447
:10410000E0EC21F012008984000EC76E220EC66E0C
:104110009E96C69E870EC96EFF0E9EB602D0E82EF2
:10412000FCD79E96C69E000EC96EFF0E9EB602D0AC
:10413000E82EFCD79E96C69E800EC96EFF0E9EB6D8
:1041400002D0E82EFCD79E96C69E800EC96EFF0E4A
:104150009EB602D0E82EFCD79E96C69E800EC96EF3
:10416000FF0E9EB602D0E82EFCD78994E0EC21F039
:1041700089849E96C69E8F0EC96EFF0E9EB602D093
:10418000E82EFCD79E96C69E010EC96EFF0E9EB607
:1041900002D0E82EFCD78994E0EC21F0120089844B
:1041A000000EC76E220EC66E9E96C69E870EC96E04
:1041B000FF0E9EB602D0E82EFCD79E96C69E000E3D
:1041C000C96EFF0E9EB602D0E82EFCD79E96C69E04
:1041D000000EC96EFF0E9EB602D0E82EFCD79E964A
:1041E000C69E800EC96EFF0E9EB602D0E82EFCD78A
:1041F0009E96C69E800EC96EFF0E9EB602D0E82E19
:10420000FCD78994E0EC21F089849E96C69E8F0E9F
:10421000C96EFF0E9EB602D0E82EFCD79E96C69EB3
:10422000010EC96EFF0E9EB602D0E82EFCD789940F
:10423000E0EC21F012008984000EC76E220EC66EDB
:104240009E96C69E8F0EC96EFF0E9EB602D0E82EB9
:10425000FCD7E0EC21F09E96C69E810EC96EFF0E43
:104260009EB602D0E82EFCD78994E0EC21F0898438
:10427000000EC76E220EC66E9E96C69E8F0EC96E2B
:10428000FF0E9EB602D0E82EFCD7E0EC21F09E9601
:10429000C69E010EC96EFF0E9EB602D0E82EFCD758
:1042A0008994E0EC21F089849E96C69E910EC96E99
:1042B000FF0E9EB602D0E82EFCD7E0EC21F09E96D1
:1042C000C69EA50EC96EFF0E9EB602D0E82EFCD784
:1042D0008994E0EC21F012008984000EC76E220E52
:1042E000C66E9E96C69E8F0EC96EFF0E9EB602D0FB
:1042F000E82EFCD7E0EC21F09E96C69E810EC96E9A
:10430000FF0E9EB602D0E82EFCD78994E0EC21F097
:1043100012008984000EC76E220EC66E9E96C69E3F
:104320008F0EC96EFF0E9EB602D0E82EFCD7E0ECD1
:1043300021F09E96C69E010EC96EFF0E9EB602D05B
:10434000E82EFCD78994E0EC21F012008984000E5D
:10435000C76E220EC66E9E96C69E910EC96EFF0E49
:104360009EB602D0E82EFCD7E0EC21F09E96C69EC9
:10437000A50EC96EFF0E9EB602D0E82EFCD789941A
:10438000E0EC21F012008984000EC76E220EC66E8A
:104390009E96C69E910EC96EFF0E9EB602D0E82E66
:1043A000FCD7E0EC21F09E96C69E000EC96EFF0E73
:1043B0009EB602D0E82EFCD78994E0EC21F01200E2
:1043C000050EE82EFED712000501256B266B276B24
:1043D000286B899A400EC76E200EC66E9E96C69EAA
:1043E000030EC96EFF0E9EB602D0E82EFCD79E9635
:1043F000C69E27C5C9FFFF0E9EB602D0E82EFCD789
:104400009E96C69E26C5C9FFFF0E9EB602D0E82E18
:10441000FCD79E96C69E25C5C9FFFF0E9EB602D04C
:10442000E82EFCD79E96C69EC952FF0E9EB602D0BD
:10443000E82EFCD7898AC950FF0A02E13AEF22F040
:10444000100E2527E86A2623E86A2723E86A28232E
:1044500005012E51130A06E005012E51170A07E047
:104460003AEF22F027A9E9EF21F03AEF22F028A154
:10447000E9EF21F0120029C500F12AC501F12BC591
:1044800002F12CC503F125C504F126C505F127C5A8
:1044900006F128C507F1C4EC1DF003BF12000501A9
:1044A0002E51130A05E005012E51170A05E01200EE
:1044B00027A960EF22F0120028A160EF22F012007D
:1044C000899A400EC76E200EC66E9E96C69E060E38
:1044D000C96EFF0E9EB602D0E82EFCD7898A899A53
:1044E0009E96C69E020EC96EFF0E9EB602D0E82EA4
:1044F000FCD79E96C69E27C5C9FFFF0E9EB602D06A
:10450000E82EFCD79E96C69E26C5C9FFFF0E9EB616
:1045100002D0E82EFCD79E96C69E25C5C9FFFF0E89
:104520009EB602D0E82EFCD79E96C69E000EC96E9F
:10453000FF0E9EB602D0E82EFCD7898A899A9E96F5
:10454000C69E050EC96EFF0E9EB602D0E82EFCD7A1
:104550009E96C69EC952FF0E9EB602D0E82EFCD78C
:10456000C9B0A8EF22F0898A0501100E2527E86A54
:104570002623E86A2723E86A28233BEF22F012006B
:10458000899A400EC76E200EC66E9E96C69E060E77
:10459000C96EFF0E9EB602D0E82EFCD7898A899A92
:1045A0009E96C69EC70EC96EFF0E9EB602D0E82E1E
:1045B000FCD7898A0501256B266B276B286B1200B7
:1045C000899A400EC76E200EC66E9E96C69E050E38
:1045D000C96EFF0E9EB602D0E82EFCD79E96C69EF0
:1045E000C952FF0E9EB602D0E82EFCD7C9CF33F5D4
:1045F000898A1200899A400EC76E200EC66E9E965A
:10460000C69EB90EC96EFF0E9EB602D0E82EFCD72C
:10461000898A1200899A400EC76E200EC66E9E9639
:10462000C69EAB0EC96EFF0E9EB602D0E82EFCD71A
:10463000898AFF0EE82EFED712000501FE0E336FA9
:104640000501000E336F2DEC1FF0ABC534F5ACC582
:1046500035F5ADC536F5AEC537F5AFC538F5B0C5DE
:1046600039F5B1C53AF50784B6C166F1B7C167F14E
:10467000B8C168F1B9C169F14BC14FF14CC150F1FA
:104680004DC151F14EC152F157C159F158C15AF1C2
:10469000079440EC14F000C13BF501C13CF502C1A8
:1046A0003DF503C13EF505015D675EEF23F05E67F2
:1046B0005EEF23F05F675EEF23F0606762EF23F049
:1046C00070EF23F05DC504F15EC505F15FC506F12D
:1046D00060C507F10101C4EC1DF003BFE0EF23F05A
:1046E00059C13FF55AC140F5B5C541F5B6C542F5CA
:1046F0000501100E326F899A400EC76E200EC66EED
:104700009E96C69E060EC96EFF0E9EB602D0E82E7D
:10471000FCD7898A899A9E96C69E020EC96EFF0EA4
:104720009EB602D0E82EFCD79E96C69E27C5C9FF2E
:10473000FF0E9EB602D0E82EFCD79E96C69E26C5DA
:10474000C9FFFF0E9EB602D0E82EFCD79E96C69EED
:1047500025C5C9FFFF0E9EB602D0E82EFCD725EE78
:1047600033F0322F02D0C0EF23F09E96C69EDECFEC
:10477000C9FFFF0E9EB602D0E82EFCD7B1EF23F0A2
:10478000898A899A9E96C69E050EC96EFF0E9EB6B0
:1047900002D0E82EFCD79E96C69EC952FF0E9EB64A
:1047A00002D0E82EFCD7C9B0CBEF23F0898A0501EF
:1047B000100E2527E86A2623E86A2723E86A2823BB
:1047C000120021C500F122C501F123C502F124C563
:1047D00003F1899A400EC76E200EC66E9E96C69E45
:1047E0000B0EC96EFF0E9EB602D0E82EFCD79E9629
:1047F000C69E02C1C9FFFF0E9EB602D0E82EFCD7AE
:104800009E96C69E01C1C9FFFF0E9EB602D0E82E3D
:10481000FCD79E96C69E00C1C9FFFF0E9EB602D071
:10482000E82EFCD79E96C69EC952FF0E9EB602D0B9
:10483000E82EFCD725EE33F00501100E326F9E9660
:10484000C69EC952FF0E9EB602D0E82EFCD7C9CF35
:10485000DEFF322F1FEF24F0898A1200899A400E62
:10486000C76E200EC66E9E96C69E900EC96EFF0E37
:104870009EB602D0E82EFCD79E96C69E000EC96E4C
:10488000FF0E9EB602D0E82EFCD79E96C69E000E66
:10489000C96EFF0E9EB602D0E82EFCD79E96C69E2D
:1048A000000EC96EFF0E9EB602D0E82EFCD79E9673
:1048B000C69EC952FF0E9EB602D0E82EFCD7C9CFC5
:1048C0002DF59E96C69EC952FF0E9EB602D0E82ECA
:1048D000FCD7C9CF2EF5898A1200B0EC1CF0B5C503
:1048E000E8FFD70802E3B0EC1CF0B5C5E8FFC80844
:1048F00002E3B0EC1CF0B5C5E8FFB90802E3B0EC88
:104900001CF0B5C5E8FFAA0802E3B0EC1CF0B5C581
:10491000E8FF9B0802E3B0EC1CF0DDEC1FF0FAECC2
:1049200022F0F29CF29E8B94899CC69AC29094824B
:10493000948C720ED36ED3A4FED789968A909390EE
:10494000FF0EE8CF00F0E82EFED7002EFCD78150F6
:10495000F294F29A9E909D909E929D92F298F2927D
:0A496000F290F286F28E0300FF00D1
:10BF0000E844F926000C160C2B0C3F0C520C640C68
:10BF1000760C860C960CA50CB30CC10CCF0CDC0C6B
:06BF2000E80CF40C000C1B
:00000001FF
